:10000000830100308A002428F60003088301CA0017
:100010008B1A0B1D1D280B11F03083120313810066
:10002000AB0AA11C1728AC0A031D1728A115211D16
:100030001D28AD0A031D1D282116031383124A082B
:100040008300F60E760E09002230840048303120FD
:1000500020308400223031208301FA2C04068001F4
:10006000840A0406031D2E28003483120313C800DB
:10007000C91B4328491B4B2849088A004808C80A5D
:100080000319C90A82008313491883174808C80A4C
:10009000840000080800FC34FE34073403340334C1
:1000A000033403340734FE34FC340F341F34383443
:1000B000303430343034303438341F340F3400347A
:1000C00008340C340E34FF34FF3400340034003470
:1000D000003400340034303430343F343F34303472
:1000E0003034003400340C340E3407340334033419
:1000F0008334C334E7347E341C34303438343C34F5
:100100003E343734333431343034303430340C34DA
:100110000E34073403340334C334E734F634BE34C6
:100120001C340C341C3438343034303430343034F3
:1001300039341F340F34FF34FF34C034C034C0347A
:10014000C034C034C034FF34FF34003400340034D1
:10015000003400340034003400343F343F347F3402
:100160007F3463346334633463346334E334C334DB
:10017000833430343034303430343034303430340C
:1001800038341F340F34FC34FE34C73463346334E2
:1001900063346334E334C73486340F341F34383463
:1001A000303430343034303438341F340F34033486
:1001B000033403348334C334E33473343B341F34A3
:1001C0000F343C343E3407340334013400340034FB
:1001D0000034003400341C34BE34F73463346334E8
:1001E00063346334F734BE341C340F341F34393471
:1001F000303430343034303439341F340F343C34FC
:100200007E34E734C334C334C334C334C734FE3418
:10021000FC340C341C343834303430343034303422
:1002200038341F340F34C034C034C034C034C03408
:10023000C034C034C034C034C0340034003400345E
:10024000003400340034003400340034003400340E
:1002500000340034003400340034003400340034FE
:1002600000340034003400340034003400340034EE
:1002700000340034003400340034003400340034DE
:1002800000340034003400340034003400343C3492
:100290003C343C343C34003400340034003400340A
:1002A0000034003400341E343F34333433343F34AC
:1002B0001E34003400340034003400340034003480
:1002C000003400340034F834FC340E340734033482
:1002D0000334033407340E340C3407341F341C3415
:1002E000383430343034303438341C340C348207F1
:1002F000C0347E3441347F34C034383444344434E0
:10030000443438347C340834103408347C340834B1
:10031000083408340834083427344834483448341E
:100320003F3440343834043404347C347C34203456
:10033000103408347C347C34403440347C34C03451
:100340002034543454345434783400340034003479
:10035000003400347F3408341434223441342234DD
:1003600049344934493436343E34413441344134DB
:100370003E347F3445344534453439347F34093490
:100380000934093406347F344834303400347F343F
:0A0390007F344934493449343634CF
:1005140002308301BE00BE0B8D2A08001230830115
:10052400BE00BE0B932A08008A308301BC00BC0BBA
:10053400992A08009E308301BC00BC0B9F2A080046
:100544008301C400861686106A238614080083017A
:10055400C000861286106A23861408008301BF0037
:100564003E0807394038A9223F087F398038A92A34
:1005740083012B08BD001930BD072B083D02BC00C8
:10058400BC08031908006400BF2AF401F501031034
:10059400F30CF20C031CD52A7008F4077108031835
:1005A400710AF5070310F00DF10D720873040319B5
:1005B4000034C92A8301BE010030B022F830BC00E7
:1005C4000130BD0064000030A222BC080319BD0341
:1005D400BC033D08803AF0008030700201300319FA
:1005E4003C02031C0800E42A6400831203138615EA
:1005F400861400008611BA2286152130A922C23041
:10060400A9220730A9221330A9222030A9220930B7
:10061400A922DC220830A9220C30A922BE01003014
:10062400B02A073083019F0086018501FF308316BD
:100634008500C430860020308B0083128C01831621
:100644008C0107308100F030831281008B17A013D6
:10065400A111A110211021122111080008308301D9
:10066400BC00BD01640005128316051200000000E1
:10067400000005168A222011051A20159022031065
:10068400BD0C201D472B8030BD078A22BC0B342BA8
:100694008A223D08080008308301BC00BD016400C3
:1006A40006118316061100000000000006158A22B8
:1006B400A0100619A01490220310BD0CA01C642BDA
:1006C4008030BD078A22BC0B512B8A223D080800CA
:1006D4008301C50064000830C600C7010612C51FA7
:1006E400752B0614762B061006160310C50DC608C6
:1006F4000319C703C6034708803AF000803070022C
:10070400013003194602031C0800702B8301BC004E
:10071400C100C2010530BF00C00101308A00410898
:100724007721BD00BE01A222C10A0319C20ABF0873
:100734000319C003BF034008803AF0008030700200
:10074400013003193F0203188F2B0030A22A8301C2
:10075400BC000830BD00A0103C18A0148312031381
:100764000611831606110000000000000000831229
:10077400A01CBF2B83160615C12B831606119022CD
:10078400831606158A220310BC0CBD0BAD2B8A2AD6
:100794008301BC000830BD0020113C1820158312D1
:1007A4000313051283160512000000000000000068
:1007B4008312201DE02B83160516E22B83160512E7
:1007C4009022831605168A220310BC0CBD0BCE2B77
:1007D4008A2A83013C08C2003D08C3000A30C000D5
:1007E400C1014308003EC90042084B3E0318C90A30
:0C07F4003520BE00BF01A222C20A03197A
:10080000C30AC0080319C103C0034108803AF000BD
:10081000803070020130031940020318F32B0030BE
:10082000A2220030A22A640083120313A301A201B2
:100830008316051606158312051206118316051276
:1008400006119C228316051606159022A011061982
:10085000A015831203132012051A20169622A01247
:100860000619A016831203132013051A2017A01AC5
:100870003B2CA201A20A201B3F2CA301A30AA01D0E
:10088000432C0230A207201E8A2A0230A3078A2A9C
:100890008301BD003C08BA00BB01BB00BA013D08A2
:1008A000BA04BB1F632C20143B08F1003A08F00087
:1008B000F009F10901307007BA0000300318013067
:1008C0007107BB00642C20100530F200F3013B08D7
:1008D000F1003A08F000C7227408AE007508AF00B6
:1008E000A501A401A6012E08B8002F08B9003908F7
:1008F000803AF000803070020A3003193802031C7D
:10090000AC2CF630380739080318390AFF3E803915
:10091000031D8F2CA60AF630B807031CB90326085E
:10092000F000F101F63E71080318710AFF3E8039AC
:10093000031D9D2CA40AF630A6072408F000F1013F
:10094000F63E71080318710AFF3E8039031D772CAB
:10095000A50AF630A407772C3808B6003908B70086
:100960002608B400B5012408B200B3012508B00080
:10097000B101201CBE2C0A30B000B101A508031D36
:100980000800A408031DF02CA608031DE52C390857
:100990003804031DD82C0B30B400B501B200350863
:1009A000B3003208B0003308B100B601B701080047
:1009B000201CDC2C0A30DD2C0B30B200B3010B30D4
:1009C000B000B101B401B5010800201CE92C0A30C7
:1009D000EA2C0B30B200B3010B30B000B1010800BB
:1009E000201CF62C0A30B000B10108000B30B0001A
:1009F000B101080064001323F622BE010030B022CA
:100A00000F3088230F3088230F3088230F3088233E
:100A10002D30882300308823053088230A3088232E
:100A20002D3088232D3088230F3088230F308823E2
:100A30000F3088230F3088230330BE000030B022EF
:100A40000F3088230F3088230F3088230F308823FE
:100A50002D30882314308823193088231E308823B2
:100A600023308823283088232D3088230F30882393
:100A70000F3088230F3088238B1313248B17220306
:100A800003195F2E2208023A0319272E8B13CC304C
:100A9000A9238B17A118532D8B134430A9238B172F
:100AA000A114AC01A111A118061D5D2DA11D5D2D84
:100AB0008B13BE30A9238B17A017BA22A01F9F2E1D
:100AC0008B134D23A7004D23A9008B17BC002708CB
:100AD0004824A111A110A013BE01BE0A0030B0220B
:100AE0001430F200F3013108F1003008F000C722A1
:100AF0007408BC007508BD00EB231430F200F3014C
:100B00003308F1003208F000C7227408BC007508F1
:100B1000BD00EB231430F200F3013508F100340876
:100B2000F000C7227408BC007508BD00EB23A508BF
:100B3000031DA62DA408031DA62DA608031DA62D82
:100B400039083804031DA62DDC30A72DF030BC0079
:100B5000BD01EB231430F200F3013708F100360831
:100B6000F000C7227408BC007508BD00EB230430F8
:100B7000BC000130BD00EB231830BC000130BD00CB
:100B8000EB230230BE000030B0221430F200F3013B
:100B90003108F1003008F000C7220A307407BC00A9
:100BA0000030031801307507BD00EB231430F2004C
:100BB000F3013308F1003208F000C7220A3074074D
:100BC000BC000030031801307507BD00EB23143062
:100BD000F200F3013508F1003408F000C7220A30B2
:100BE0007407BC000030031801307507BD00EB230B
:100BF000A508031D072EA408031D072EA608031D24
:100C0000072E39083804031D072EE630082EFA3067
:100C1000BC00BD01EB231430F200F3013708F100F2
:100C20003608F000C7220A307407BC0000300318F1
:100C300001307507BD00EB230E30BC000130BD0054
:100C4000EB232230BC000130BD00EB239F2EBE0100
:100C5000BE0A0030B0222D3088232D3088232D305D
:100C600088232D3088232D3088232D3088232D3064
:100C700088232D3088232D3088232D3088232D3054
:100C800088232D3088232D3088232D30882302306F
:100C9000BE000030B0222D3088232D3088232D3027
:100CA00088230F3088233C30882341308823463006
:100CB00088234B308823503088230F30962EBE0176
:100CC000BE0A0030B0222D3088232D3088232D30ED
:100CD00088232D3088232D3088232D3088232D30F4
:100CE00088232D3088232D3088232D3088232D30E4
:100CF00088232D3088232D3088232D3088230230FF
:100D0000BE000030B0222D3088232D3088232D30B6
:100D100088232D3088232D3088230F3088233230CC
:100D20008823373088230F3088232D3088232D30B7
:100D300088232D3088232D3088232D3088232303CA
:100D40000319BF2F2308023A0319872F8B13CC30C6
:100D5000CA238B172119B32E8B134430CA238B1748
:100D60002115AD0121122119051EBD2E211EBD2EFA
:100D70008B13BE30CA238B172114BA22211CFD2CE1
:100D80008B133023A8003023AA008B17BC0028083F
:100D900048242112211121100430BE000030B0225D
:100DA0001430F200F3013108F1003008F000C722DE
:100DB0007408BC007508BD00EB231430F200F30189
:100DC0003308F1003208F000C7227408BC0075082F
:100DD000BD00EB231430F200F3013508F1003408B4
:100DE000F000C7227408BC007508BD00EB23A508FD
:100DF000031D062FA408031D062FA608031D062F9A
:100E000039083804031D062FDC30072FF030BC00F2
:100E1000BD01EB231430F200F3013708F10036086E
:100E2000F000C7227408BC007508BD00EB23043035
:100E3000BC000130BD00EB231830BC000130BD0008
:100E4000EB230530BE000030B0221430F200F30175
:100E50003108F1003008F000C7220A307407BC00E6
:100E60000030031801307507BD00EB231430F20089
:100E7000F3013308F1003208F000C7220A3074078A
:100E8000BC000030031801307507BD00EB2314309F
:100E9000F200F3013508F1003408F000C7220A30EF
:100EA0007407BC000030031801307507BD00EB2348
:100EB000A508031D672FA408031D672FA608031D9F
:100EC000672F39083804031D672FE630682FFA3082
:100ED000BC00BD01EB231430F200F3013708F10030
:100EE0003608F000C7220A307407BC00003003182F
:100EF00001307507BD00EB230E30BC000130BD0092
:100F0000EB232230BC000130BD00EB23FD2C04306C
:100F1000BE000030B0222D3088232D3088232D30A4
:100F200088232D3088232D3088232D3088232D30A1
:100F300088232D3088232D3088232D3088232D3091
:100F400088232D3088232D3088232D3088230530A9
:100F5000BE000030B0222D3088232D3088232D3064
:100F600088230F3088233C30882341308823463043
:100F700088234B308823503088230F30F62F0430DD
:100F8000BE000030B0222D3088232D3088232D3034
:100F900088232D3088232D3088232D3088232D3031
:100FA00088232D3088232D3088232D3088232D3021
:100FB00088232D3088232D3088232D308823053039
:100FC000BE000030B0222D3088232D3088232D30F4
:100FD00088232D3088232D3088230F30882332300A
:100FE0008823373088230F3088232D3088232D30F5
:100FF00088232D3088232D3088232D308823FD2C05
:02400E003C3F35
:00000001FF
